:02000000002AD4
:020008000900ED
:100020008207FE34C8349634643450344334353453
:10003000293421341B3415340F340A34083406347F
:1000400004348207643450343C342D342634213453
:100050001E341B34153411340E340A34073405347D
:100060000434043482070134013402340434043487
:10007000043408340834083408341034103410348C
:1000800020344034403482070134013402340434D3
:10009000063408340C341034143418342034283422
:1000A000303440348034DF3482070834043402347E
:0A00B0000134083404340234013432
:1001C0008A01CF03031D08000A30CF000F304E050F
:1001D0008207372E3A2E372E422E372E4A2E372EB2
:1001E000792E522E372E5A2E372E622E6A2E792EC7
:0201F000792E66
:1002000082070834043402340134083404340234DC
:100210000134013402340434083401340234043427
:100220000834013402340434083408340434023409
:100230000134013402340434083404340234013407
:1002400004340C340634033409340C3406340334D7
:100250000934033406340C340934033406340C34C2
:100260000934033406340C34093409340C340634AC
:100270000334033406340C3409340C3406340334A8
:10028000093407340E340D340B3407340E340D3476
:100290000B3407340E340D340B3407340E340D3464
:1002A0000B3407340B340D340E340E340D340B3450
:1002B000073407340B340D340E340D340B3407344B
:1002C0000D34003408340C340E340F340734033446
:1002D000013400340134033407340F340E340C3449
:1002E0000834003408340C340E340F340E340C341B
:1002F000083408340C340E34073403340134023427
:1003000004340C3403340C3403340C3403340C3410
:100310000334093406340934063409340634093404
:1003200006340A3405340A3405340A3405340A34F0
:1003300005340A3405340A3405340C3403340C34DF
:1003400003340F34003400340034003400340034FB
:1003500000340F340034003400340F3400340034DF
:1003600000340F3400340F340034003400340034CF
:1003700000340F3400340F3400340F3400340F34A1
:10038000003408340434023401340C340E340F3495
:1003900002340F34003400340034013402340434A5
:1003A000083408340F3404340F3402340F34013469
:1003B0000F34063409340234043403340C34023468
:1003C0000134083402340434063409340234063467
:1003D0000E34013405340A3405340A340734023447
:1003E0000E34083408340434043402340234013442
:1003F000013408340834043404340234023404343C
:100400008316FF308700FF308800073089000730EF
:100410009F000730810083018316FF308500FF3085
:100420008600A0308700F030880007308900003057
:10043000810000309F008301831620308C009901D9
:100440002230980064008301903098008C018B0169
:100450008B0164008301203084008001840A040839
:10046000803C031D2D2AA03084008001840A0408EA
:10047000F03C031D352A8317103084008001840A64
:100480000408703C031D3E2A903084008001840AD9
:100490000408F03C031D462A640083010130C200B9
:1004A0000130C3000730B4000C30B8000030D10078
:1004B0000330D2000130D400D0010130D300071442
:1004C00054186F2AE020FF30BA00FF30BB00FF3025
:1004D000BC00FF30BD000026EE260927602A541C10
:1004E000602A00267B260927EE26E0205208003CE1
:1004F0000319A92AD703031D6F2A9630D700D60304
:10050000031D6F2A3208D600871C882A8710892A83
:1005100087145208013C03199E2A5208023C031911
:10052000922AEA2A07158711B60A7F30B6053608DF
:100530000A150A1400258A01B9006F2A07118715C8
:10054000B60A7F30B60536080A1500248A01B900BC
:100550006F2AD703031D6F2AFA30D70007118711BE
:10056000C20A4208053C031DD52AC201C30A43083A
:1005700044020318D52AC301871CC02A8710C12A48
:100580008714B01CCA2AB8033808003C031DD02ABF
:10059000B010D02AB80A38080F3C031DD02AB01476
:1005A00038080F392120C5006F2A6400C103031DDC
:1005B0006F2A4508C100B01CDF2AB403E02AB40A40
:1005C0000730B40534085420B90038080F394320E7
:1005D000B5006F2A071587155108073C031DF52A3A
:1005E0005008033C031DF52AD0015108B600B60E91
:1005F000B60DE030B6055008B700B70DB70D370D92
:100600001839B604B40A0730B4053408B6073608FA
:0A0610000A1400218A01B9006F2AC4
:1008000082070134023404340834013402340434DD
:10081000083401340234043408340134023404341A
:1008200008340C340C340C340634063406340334E7
:10083000033403340934093409340C340C340C34D3
:1008400000340F340034003400340F3400340034EA
:1008500000340F340E340C340834013403340734BC
:100860000E34063402340F3400340F3400340F34A5
:1008700000340834043402340134083404340234BB
:1008800001340834043402340134083404340234AA
:10089000013408340434023401340234043408349A
:1008A000013402340434083401340234043408348A
:1008B00001340234043408340C340E340F34073459
:1008C0000334013408340C340E340F340734033449
:1008D000013400340F3400340E3400340C3400344E
:1008E00008340C340634033409340C34063403342D
:1008F00009340C340634033409340C34063403341C
:1009000009340C34033403340C340C34033403340E
:100910000C340C34033403340C340C3403340334FB
:100920000C340634093406340934063409340634E8
:1009300009340634093406340934063409340F34D2
:100940000034003400340034003400340034003407
:1009500000340034003400340034003400340034F7
:1009600000340034003400340034003400340034E7
:1009700000340034003400340034003400340034D7
:1009800000340034003400340034003400340034C7
:1009900000340034003400340034003400340034B7
:1009A00000340034003400340034003400340034A7
:1009B0000034003400340034003400340034003497
:1009C0000034003400340034003400340034003487
:1009D0000034003400340034003400340034003477
:1009E0000034003400340034003400340034003467
:1009F0000034003400340034003400340034003457
:100A000082070134043402340834013403340734D7
:100A10000F340E340C3408340F3400340F340634E1
:100A2000023401340834043402340134023404340E
:100A300008340C340E340F340734033409340C34C6
:100A40000634033409340C340634093406340934CA
:100A500006340F3406340F340734033401340834B9
:100A600004340234043402340834013404340234CB
:100A700008340F3400340F3400340F34003406349B
:100A8000003409340C3403340C3406340334063493
:100A90000C34003403340C340E3407340B340D346E
:100AA0000E3407340334013408340434023401347E
:100AB000023404340834093404340E340F34073457
:100AC0000334013408340C340E340F340734033447
:100AD000013400340F3400340E3400340C3400344C
:100AE00008340C340634033409340C34063403342B
:100AF00009340C340634033409340C34063403341A
:100B000009340C34033403340C340C34033403340C
:100B10000C340C34033403340C340C3403340334F9
:020B20000C3493
:100C0000D803031D08004008003C0319092EC00347
:100C10000800861E2B2E861F212E061F272E061E3D
:100C2000312E061D1B2E861D162E08006430C000B6
:100C3000D401871008006430C0000130D40087144C
:100C400008006430C000D00A0330D00508006430CA
:100C5000C000D30A08006430C000D20A0330D205B5
:100C600008006430C000D10A0730D1050800CE0A60
:100C70001F1508001F190800CE0A1E08CB00C93036
:100C80009F0008001F190800CE0A1E08CD00D130B1
:100C90009F0008001F190800CE0A1E08CC00E13092
:100CA0009F0008001F190800CE0A1E08C800E9307E
:100CB0009F0008001F190800CE0A1E08C900F13065
:100CC0009F0008001F190800CE0A1E08CA00F9304C
:100CD0009F000800CE0A4D08C400C4090330C404B4
:100CE0004D0E0F391020B2004D0E0F393220B500D5
:100CF0000800CE0A0800D903031D0800FA30D90005
:100D0000531CE02E07103918902E3A08033C0318A4
:100D10009A2E3508BA0203189A2E0330BA009A2E7A
:100D20003A08F73C031C9A2E3508BA07031C9A2E82
:100D3000FA30BA00B918A72E3B08033C0318B12EAD
:100D40003508BB020318B12E0330BB00B12E3B089F
:100D5000F73C031CB12E3508BB07031CB12EFA303B
:100D6000BB003919BE2E3C08033C0318C82E3508B9
:100D7000BC020318C82E0330BC00C82E3C08F73C48
:100D8000031CC82E3508BC07031CC82EFA30BC0053
:100D9000B919D52E3D08033C0318DF2E3508BD02D6
:100DA0000318DF2E0330BD00DF2E3D08F73C031C87
:100DB000DF2E3508BD07031CDF2EFA30BD0008000A
:100DC0000714BA013918BA03BB01B918BB03BC0137
:100DD0003919BC03BD01B919BD0308006400B10392
:100DE0000319042F31085B020319881031085C02D3
:100DF0000319081031085D020319881131085E02D9
:100E000003190712830108008814081488150716AF
:100E10000800DA03031D0800D50A56275508013CCF
:100E20000319272F5508023C03192F2F5508033C9F
:100E30000319372F5508043C03193F2F5508053C6B
:100E40000319242FD5010800FF30990008003A0843
:100E5000A1004808A2005C272308DB00472F3B08BD
:100E6000A1004908A2005C272308DC00472F3C08AA
:100E7000A1004A08A2005C272308DD00472F3D0897
:100E8000A1004B08A2005C272308DE00472F23089F
:100E9000A1004C08A2005C272308FF3C031D532F30
:100EA000FE309900080023089900080083166400AA
:100EB000981C572F83120800A301A40122080310D5
:100EC0002118A307A30CA40CA118A307A30CA40C1E
:100ED0002119A307A30CA40CA119A307A30CA40C0C
:100EE000211AA307A30CA40CA11AA307A30CA40CFA
:100EF000211BA307A30CA40CA11BA307A30CA40CE8
:020F00000800E7
:021000000000EE
:02400E00060D9D
:00000001FF
